:020000040000FA
:1000000025000400930C0200080C0600660078002E
:10001000700076004B0C370066071A0AF6020C0ACD
:10002000F7020C0A50053006780058043004180214
:1000300026000C0A580CB3091006C70A150C240038
:10004000070C90091006C70A140C2400050C90092F
:100050001006C70A030C3300060CB3091006C70AC2
:10006000F3022C0A030435033403340314031F0E74
:100070003400010F43075E0A50075E0A1502000FA5
:1000800043066F0A1502010F4306740A1502030F97
:100090004306790A1502040F43067B0A1502090F6D
:1000A0004306850A1502080F4306830A1502060F48
:1000B0004306670A1502070F43066B0A15029A01E9
:1000C00043070C0A1402990143070C0A090A050C9C
:1000D00038003005880A060C38003005880A010C03
:1000E000B80118065805880A020CB80138065805E8
:1000F000880A1804880A3804880A050C3800880A17
:10010000060C3800880A7800880A070C3800880A2C
:100110001802260050041402390015023A00090A98
:100120003300B50CA00910060008C80CB30910066E
:1001300000080304660703052003F302910A000880
:1001400021000602080E320010040602080E3100DB
:1001500092015201430700081102320001024307D5
:10016000A50A1005000821000602080E320010043E
:100170000602080E3100920152014307C50A11021E
:100180003200010243060008B80A10050008010CFD
:10019000210001024307C90A0C0A700869086308B4
:1001A000700872086F086A086508630874087308A5
:1001B0002E086F08720867082E0875086B0820085B
:1001C0002808430829082008320830083108300878
:0A01D0002008760831082E083508D3
:021FFE00EB0FE7
:00000001FF
